:020000040000FA
:040000006F303A28FB
:08000800A000030EA100831209
:1000100081018B100B11210E8300A00E200E090010
:0C007400203084008001840A6030040207
:10008000031C3C281230B0007C2183160C308505FF
:1000900087018312850187010730990000309A009B
:1000A000103083168E008312603083168F00831207
:1000B0000030831691008312C830831681008312AA
:1000C00031309000003083168C00831210308B008A
:1000D000831600309B001C141A088312BC00831680
:1000E00010309B001C141A088312BD00AA2183162D
:1000F00020309B001C141A088312C2000130C20871
:100100000319C20081018E018F010B118B100B109E
:100110008C018B179A2031199C205E21B30B9828F3
:10012000031085190314B90DF03039020319BA21EF
:10013000C6218A2864000800080031110130B70088
:100140008B132030370783169B001C141A08831268
:10015000A4001030370783169B001C141A08831262
:10016000A3000030370783169B001C141A08831263
:10017000A2008B17321CC22822090339A200A3094E
:10018000A409A50901303702031DCB283D18CB284F
:100190003D143E14832102303702031DD428BD18BC
:1001A000D428BD143E148C2103303702031DDD28F2
:1001B0003D19DD283D153E14952104303702031DFD
:1001C000E628BD19E628BD153E149E2105303702EC
:1001D000031DEF283D1AEF283D163E14A6210630D8
:1001E0003702031DF828BD1AF828BD163E14A721B2
:1001F00007303702031D01293D1B01293D173E141D
:10020000A82108303702031D0A29BD1B0A29BD1782
:100210003E14A921B70A0530370203180800A028A8
:100220000130B600B300B400B500B7008501870106
:10023000B1139A20B30B3629031085190314B90D95
:10024000F030390203195429B41F8501B41F870106
:10025000B40B36293708B6080319B6000319342938
:10026000FF3085008700B6039630B400311D192990
:100270003111321C40292D090339AD00AE09AF09F7
:100280008B1320303707BB002F08BA0067211030CE
:100290003707BB002E08BA00672100303707BB00C4
:1002A0002D08BA0067218B1785018701B70AB601AF
:1002B00005303702031C1929AA2108003E1C08003A
:1002C0003E101030BB003D08BA00672108008B13B8
:1002D0003A0883161C159A0083123B0883169B006C
:1002E00055309D00AA309D009C1464009C1875290F
:1002F0001C1183128B1708000130D500D200EE309C
:10030000D000D10008000130D500D200EE30D0007E
:10031000D1000130BD0008000130D500D200EE3020
:10032000D000D1000230BD0008000130D500D2005D
:10033000EE30D000D1000430BD0008000130D500FF
:10034000D200EE30D000D100BD0108000800080046
:100350000800080001303D020319080002303D0288
:100360000319080004303D02031908000130BD00E4
:100370003E1408003E140310BD0D0130D500D2001C
:10038000EE30D000D100BD193D1408008F080319CC
:1003900008008F01C10B08004208C100D50B0800FE
:1003A0005608D50007303D050319FD29D21BD00A98
:1003B000D21FD0030A305002031CF829D0010930A3
:1003C000D21FD0005203D2007F39031DF829D10A71
:1003D00010305102031CED29D1015022D2006022BD
:1003E000D4007022D600D500D0010930D21FD00031
:1003F0000023850024238700080085018701080069
:1004A00002308A0051083D1C572A883E8200BD1C3C
:1004B0005B2A883E82003D1D5F2A983E8200003400
:1004C00002308A0051083D1C672AA83E8200BD1CEC
:1004D0006B2AB83E82003D1D6F2AB83E8200003470
:1004E00002308A0051083D1C772AC83E8200BD1C9C
:1004F0007B2AD83E82003D1D7F2AE83E82000134DF
:100510000734873407348734033483340334833413
:100520000B3403340F3407340B34033403340734EF
:10053000053487340734253483340334073489344D
:100540000B3403348F3405348B34113403340334C7
:1005500001340134023402340434043408340834DD
:10056000103410342034203440344034803480340B
:10057000083404340234803440348034103402347B
:10058000043410342034013404344034843480344E
:10059000093409340A340A34083408340834083475
:1005A0000834183408341834083418341034083433
:1005B000093429340A341A34283408340834083405
:1005C0000A34383408341A3408345834103448346F
:1005D000293409340A340A342834083408344834B5
:1005E0002834183488341834283418341034083433
:1006000003308A005008541C072B4B3E8200D41C38
:100610000B2B563E8200541D0F2B613E8200D41DD1
:10062000132B6C3E8200541E172B773E8200D41E83
:100630001B2B823E8200541F1F2B8D3E8200D41F35
:10064000232B983E8200003403308A005008541C4B
:100650002B2BA33E8200D41C2F2BAE3E8200541DB8
:10066000332BB93E8200D41D372BC43E8200541E6A
:100670003B2BCF3E8200D41E3F2BDA3E8200541F1C
:10068000432BE53E8200D41F472BF03E820000340E
:0A0696001034203401340234003423
:0A06A000003400340034003400344C
:0406AC0010343034A2
:1006B0003134333433343334333433343334333404
:0E06C2000034003400340034003400340234BC
:0606D0000334233433342F
:0806D800103420340134023417
:0C06E000003410342034013402340034A3
:0206EE001034C6
:1006F0002034013402340034003402340134203414
:020700001034B3
:0C070400103430343134333433343334A7
:080710003134303410340034A0
:06071A00333423340334E4
:0E072000023400340034023403342334333402
:10073000333400343334003433340034333400344D
:04074000333400341A
:0A07460000340034003400340234A3
:0A075000043401342034103408345E
:04075C000034003431
:1007600000340034023406340734273437343F343D
:0E07720008341834383439343D343F343F34C1
:060780003F343F343F341A
:08078800043401342034103464
:0C0790000A3404340134203410340A34DC
:02079E0008341D
:1007A000103420340134063406340134203410343B
:0207B00008340B
:0C07B40008341834383439343F343934F8
:0807C000383418340834003409
:0607CA003F3437342734F0
:0E07D0000734063406340734273437343F34F8
:1007E0003F3400343F3400343F3400343F3400346D
:0407F0003F3400345E
:084000000C00030002000600A1
:02400E00CC33B1
:10420000FF00FF00FF00FF00FF00FF00FF00FF00B6
:10421000FF00FF00FF00FF00FF00FF00FF00FF00A6
:104220000100FF00FF00FF00FF00FF00FF00FF0094
:10423000FF00FF00FF00FF00FF00FF00FF00FF0086
:104240001000FF00FF00FF00FF00FF00FF00FF0065
:10425000FF00FF00FF00FF00FF00FF00FF00050060
:10426000FF00FF00FF00FF00FF00FF00FF00FF0056
:10427000FF00FF00FF00FF00FF00FF00FF00FF0046
:10428000FF00FF00FF00FF00FF00FF00FF00FF0036
:10429000FF00FF00FF00FF00FF00FF00FF00FF0026
:1042A000FF00FF00FF00FF00FF00FF00FF00FF0016
:1042B000FF00FF00FF00FF00FF00FF00FF00FF0006
:1042C000FF00FF00FF00FF00FF00FF00FF00FF00F6
:1042D000FF00FF00FF00FF00FF00FF00FF00FF00E6
:1042E000FF00FF00FF00FF00FF00FF00FF00FF00D6
:1042F000FF00FF00FF00FF00FF00FF00FF000000C5
:00000001FF
